:10000000B0C00000CAC00000C8C00000C6C00000E8
:10001000C4C00000C2C00000C0C00000BEC00000DC
:10002000BCC00000BAC00000B8C00000B6C00000EC
:10003000B4C00000B2C00000B0C00000AEC00000FC
:10004000ACC00000AAC00000A8C00000A6C000000C
:10005000A4C00000A3C00000A0C000009EC000001B
:100060009CC000009AC0000000407A10F35A00A023
:10007000724E18090010A5D4E80000E87648170071
:1000800000E40B54020000CA9A3B000000E1F505B1
:10009000000080969800000040420F000000A086FB
:1000A00001000000102700000000E803000000002D
:1000B0006400000000000A000000000001000000D1
:1000C00000002C76D888DC674F0823DFC1DFAE59EB
:1000D000E1B1B796E5E3E453C63AE651997696E87E
:1000E000E6C28426EB898C9B62ED407C6FFCEFBC02
:1000F0009C9F40F2BAA56FA5F490055A2AF75C932D
:100100006B6CF9676DC11BFCE0E40D47FEF520E662
:10011000B500D0ED902E0300943577050080841E45
:10012000080000204E0A000000C80C333333330FA0
:10013000986E12831141EF8D2114893BE65516CF3D
:10014000FEE6DB18D1844B381BF77C1D901DA4BB49
:10015000E424203284725E228100C9F124ECA1E5FE
:100160003D2711241FBECFEFD8E0DEBFCDBF11E089
:10017000A0E0B1E0E8E4F7E102C005900D92A639F5
:10018000B107D9F721E0A6E9B1E001C01D92A23A7A
:10019000B207E1F7D8D20C94A20B32CF1895ECE756
:1001A000F0E0808180648083EAE7F0E08081846011
:1001B0008083808180688083089583B7817F826097
:1001C00083BFEAE7F0E080818860808378940895B7
:1001D0002F923F924F925F926F927F928F929F9257
:1001E000AF92BF92CF92DF92EF92FF920F931F9345
:1001F000CF93DF93CDB7DEB7CA55D1090FB6F894C8
:10020000DEBF0FBECDBF982E892E68966FAF689760
:1002100069967FAF6997742E622E17012801C60177
:10022000B5016E012AE4C20ED11C860123E045E02F
:100230006B963FAF6B976A965FAF6A9741D55E0149
:100240008DE3A80EB11C850123E045E0C201B10198
:1002500037D56A965FAD6A975F937F926B963FAD95
:100260006B973F936F928F929F9269969FAD69971C
:100270009F9368962FAD68972F9380E091E09F93AE
:100280008F931F9288E28F930C5311091F930F9342
:1002900037D5BF92AF92DF92CF928CE191E09F93DE
:1002A0008F931F9284E18F936E0189E2C80ED11C57
:1002B000DF92CF9225D5C80174D2C60172D20FB693
:1002C000F894DEBF0FBECDBFC65ADF4F0FB6F8940D
:1002D000DEBF0FBECDBFDF91CF911F910F91FF9079
:1002E000EF90DF90CF90BF90AF909F908F907F90D6
:1002F0006F905F904F903F902F90089590917C0069
:10030000907F982B90937C0020E130E080E090E09B
:10031000DC0143B7416043BF889543B74E7F43BF7D
:100320004091780050917900840F951FA11DB11D57
:10033000215031092115310561F79C01AD0182E0A1
:1003400056954795379527958A95D1F7A2EFB2E153
:100350003AD22CE096958795779567952A95D1F7AF
:10036000695F7F4F8F4F9F4F49D317D3CB010895BC
:10037000CF92DF92EF92FF926B017C0120E030E0A0
:10038000A9019FD287FD0BC020E030E040EA50E495
:10039000C701B6019AD24BD400D3CB0102C080E092
:1003A00090E0FF90EF90DF90CF900895CF92DF9292
:1003B000EF92FF926B017C0120E030E84CED53E4BA
:1003C00080D287FD10C020E030E84CED53E4C70137
:1003D000B60112D220E030E048E151E476D227D4D1
:1003E000DCD2CB0102C080E090E0FF90EF90DF9084
:1003F000CF9008952F923F924F925F926F927F928B
:100400008F929F92AF92BF92CF92DF92EF92FF9224
:100410000F931F93CF93DF936B017C0120E030E0BB
:1004200040E850E44ED287FD74C020E030E04CE557
:1004300054E4C701B60194D318160CF46FC041E41C
:10044000A42E41E0B42E00E010E0E8012196F50171
:1004500060817181882777FD8095982FD1D2A7017F
:1004600096017ED3181644F0F6E0AF0EB11CCE30E4
:10047000D10519F08E01E9CFE8018E010F5F1F4F02
:1004800036E0732E7C9EF0017D9EF00D1124E55C1C
:10049000FE4FC081D18182809380A480B580BE014F
:1004A000882777FD8095982FABD29B01AC01C701BF
:1004B000B601A2D11B012C01709E7001719EF00C3F
:1004C0001124C701855C9E4F7C01A5019401FC01AC
:1004D00062817381848195818FD19B01AC01C201BE
:1004E000B10142D32B013C01F701608171816C1B8A
:1004F0007D0B882777FD8095982F82D29B01AC01D8
:10050000C301B201E2D19B01AC01C501B40175D1B7
:1005100009C060E070E080E090E404C06DEC7CEC29
:100520008CE49FE3DF91CF911F910F91FF90EF90AB
:10053000DF90CF90BF90AF909F908F907F906F9003
:100540005F904F903F902F9008952F923F924F923F
:100550005F926F927F928F929F92AF92BF92CF9253
:10056000DF92EF92FF920F931F93CF93DF93CDB75C
:10057000DEB72C970FB6F894DEBF0FBECDBF6983F0
:100580007A838B839C8329873A874B875C87F0DE4D
:100590001C0129853A854B855C85CA01B90106DFB6
:1005A0004C01C801B70126DF5B016C0129853A8542
:1005B0004B855C85CA01B901F0D16D837E838F8341
:1005C000988769817A818B819C81E7D1DC01CB019D
:1005D00094014D815E81B101FBDD2C960FB6F8943C
:1005E000DEBF0FBECDBFDF91CF911F910F91FF9066
:1005F000EF90DF90CF90BF90AF909F908F907F90C3
:100600006F905F904F903F902F900895CF92DF9220
:10061000EF92FF920F931F9382E090E06FDEBC0198
:10062000882777FD8095982FEBD120E030E040E3DC
:1006300051E44BD16B017C0160919E0170919F014F
:100640008091A0019091A1019B01AC01D6D09B01AA
:10065000AC01C701B601D1D020E030E040E450E465
:1006600034D160939E0170939F018093A001909379
:10067000A10185E090E042DEBC01882777FD8095EE
:10068000982FBED16B017C0160919A0170919B0102
:1006900080919C0190919D019B01AC01AED09B018A
:1006A000AC01C701B601A9D020E030E040E450E43D
:1006B0000CD160939A0170939B0180939C0190935D
:1006C0009D0180E090E01ADEBC01882777FD8095CF
:1006D000982F96D16B017C016091960170919701E2
:1006E00080919801909199019B01AC0186D09B016A
:1006F000AC01C701B60181D020E030E040E450E415
:10070000E4D09B01AC0160939601709397018093B4
:10071000980190939901E0909E01F0909F010091C3
:10072000A0011091A10160919A0170919B018091AB
:100730009C0190919D0109DF1F910F91FF90EF9017
:10074000DF90CF90089515D02ADD37DDE12CF12C14
:100750008701A8019701C801B701F7DE57DF2FE332
:100760008DE093E0215080409040E1F700C0000010
:10077000F5CF1092C5008CE08093C400E0ECF0E06F
:1007800080818260808388E18093C10086E08093CD
:10079000C20008959091C00095FFFCCF8093C600E1
:1007A00008951F93CF93DF93EC0110E0FE01E10F5A
:1007B000F11D8081882319F0EDDF1F5FF7CFDF91F6
:1007C000CF911F91089509D0A59F900DB49F900DD2
:1007D000A49F800D911D11240895A29FB001B39F85
:1007E000C001A39F700D811D1124911DB29F700D3A
:1007F000811D1124911D08955058BB27AA270ED0A2
:1008000075C166D130F06BD120F031F49F3F11F407
:100810001EF45BC10EF4E095E7FB51C1E92F77D1DF
:1008200080F3BA17620773078407950718F071F40D
:100830009EF58FC10EF4E0950B2EBA2FA02D0B0163
:10084000B90190010C01CA01A0011124FF27591B15
:1008500099F0593F50F4503E68F11A16F040A22F1B
:10086000232F342F4427585FF3CF4695379527958C
:10087000A795F0405395C9F77EF41F16BA0B620B8B
:10088000730B840BBAF09150A1F0FF0FBB1F661FD2
:10089000771F881FC2F70EC0BA0F621F731F841F15
:1008A00048F4879577956795B795F7959E3F08F03B
:1008B000B3CF9395880F08F09927EE0F97958795FA
:1008C0000895D9D008F481E008950CD00FC107D164
:1008D00040F0FED030F021F45F3F19F0F0C051112C
:1008E00039C1F3C014D198F39923C9F35523B1F357
:1008F000951B550BBB27AA2762177307840738F08F
:100900009F5F5F4F220F331F441FAA1FA9F333D0ED
:100910000E2E3AF0E0E830D091505040E695001CA1
:10092000CAF729D0FE2F27D0660F771F881FBB1F5D
:10093000261737074807AB07B0E809F0BB0B802D37
:10094000BF01FF2793585F4F2AF09E3F510568F083
:10095000B6C000C15F3FECF3983EDCF38695779517
:100960006795B795F7959F5FC9F7880F911D969585
:10097000879597F90895E1E0660F771F881FBB1FE1
:10098000621773078407BA0720F0621B730B840B8E
:10099000BA0BEE1F88F7E095089504D06894B11162
:1009A000D9C00895BCD088F09F5790F0B92F9927EF
:1009B000B751A0F0D1F0660F771F881F991F1AF06A
:1009C000BA95C9F712C0B13081F0C3D0B1E0089533
:1009D000C0C0672F782F8827B85F39F0B93FCCF3B4
:1009E000869577956795B395D9F73EF49095809560
:1009F000709561957F4F8F4F9F4F0895E89409C080
:100A000097FB3EF490958095709561957F4F8F4F41
:100A10009F4F9923A9F0F92F96E9BB279395F69557
:100A2000879577956795B795F111F8CFFAF4BB0FD5
:100A300011F460FF1BC06F5F7F4F8F4F9F4F16C039
:100A4000882311F096E911C0772321F09EE8872FC3
:100A5000762F05C0662371F096E8862F70E060E07F
:100A60002AF09A95660F771F881FDAF7880F9695F8
:100A7000879597F90895990F0008550FAA0BE0E89C
:100A8000FEEF16161706E807F907C0F01216130650
:100A9000E407F50798F0621B730B840B950B39F490
:100AA0000A2661F0232B242B252B21F408950A26F6
:100AB00009F4A140A6958FEF811D811D089597F936
:100AC0009F6780E870E060E008959FEF80EC0895F4
:100AD00000240A941616170618060906089500241D
:100AE0000A9412161306140605060895092E039497
:100AF000000C11F4882352F0BB0F40F4BF2B11F40B
:100B000060FF04C06F5F7F4F8F4F9F4F089557FD69
:100B10009058440F551F59F05F3F71F04795880F6B
:100B200097FB991F61F09F3F79F087950895121602
:100B300013061406551FF2CF4695F1DF08C01616AE
:100B400017061806991FF1CF86957105610508945F
:100B50000895E894BB2766277727CB0197F9089576
:100B60008ADF08F48FEF08950BD0C0CFB1DF28F0F3
:100B7000B6DF18F0952309F0A2CFA7CF1124EACF52
:100B8000C6DFA0F3959FD1F3950F50E0551F629FEC
:100B9000F001729FBB27F00DB11D639FAA27F00DD6
:100BA000B11DAA1F649F6627B00DA11D661F829FFD
:100BB0002227B00DA11D621F739FB00DA11D621FE2
:100BC000839FA00D611D221F749F3327A00D611DFF
:100BD000231F849F600D211D822F762F6A2F1124E1
:100BE0009F5750408AF0E1F088234AF0EE0FFF1F34
:100BF000BB1F661F771F881F91505040A9F79E3F6B
:100C0000510570F05CCFA6CF5F3FECF3983EDCF36C
:100C1000869577956795B795F795E7959F5FC1F7A7
:100C2000FE2B880F911D9695879597F9089577DF8C
:100C3000E0F09E37D8F09639B8F49E3848F4672F24
:100C4000782F8827985FF9CF869577956795939544
:100C50009539D0F3B62FB1706B0F711D811D20F443
:100C6000879577956795939502C01CC073CF8823AD
:100C700071F4772321F09850872B762F07C06623D5
:100C800011F499270DC09051862B70E060E02AF096
:100C90009A95660F771F881FDAF7880F96958795C4
:100CA00097F908959F3F31F0915020F487957795FB
:100CB0006795B795880F911D9695879597F9089533
:100CC000EF920F931F93CF93DF93E80147FF02C08A
:100CD00034E101C034E0E42FFF27E7FDF095F7FF92
:100CE00003C0F195E195F109E32E022F2E2FAE01FD
:100CF000F7D1CE01DF91CF911F910F91EF90089521
:100D0000AEE0B0E0E5E8F6E0F4C40D891E898F8915
:100D1000988D26E02C831A83098397FF02C080E018
:100D200090E801979E838D83AE01455E5F4F698D8C
:100D30007A8DCE01019611D04D815E8157FD0AC09A
:100D40002F813885421753070CF49A01F801E20FFE
:100D5000F31F10822E96E4E0E8C4ACE0B0E0E2EBD2
:100D6000F6E0B9C47C016B018A01FC01178216828E
:100D7000838181FFB0C1CE0101964C01F7019381BF
:100D8000F60193FD859193FF81916F01882309F40A
:100D90009EC1853239F493FD859193FF81916F0156
:100DA000853221F4B70190E006D4E8CF512C312CE4
:100DB00020E02032A0F48B3269F030F4803259F018
:100DC000833269F420612CC08D3239F0803339F4DC
:100DD000216026C02260246023C0286021C027FD36
:100DE00027C030ED380F3A3078F426FF06C0FAE01D
:100DF0005F9E300D1124532E13C08AE0389E300DB3
:100E00001124332E20620CC08E3221F426FD5FC1E6
:100E1000206406C08C3611F4206802C0883641F484
:100E2000F60193FD859193FF81916F018111C1CFEF
:100E3000982F9F7D9554933028F40C5F1F4FFFE34C
:100E4000F9830DC0833631F0833771F0833509F0B3
:100E500057C021C0F801808189830E5F1F4F442451
:100E60004394512C540114C03801F2E06F0E711CF0
:100E7000F801A080B18026FF03C0652D70E002C09C
:100E80006FEF7FEFC5012C878BD32C0183012C855D
:100E90002F77222E16C03801F2E06F0E711CF80178
:100EA000A080B18026FF03C0652D70E002C06FEF07
:100EB0007FEFC5012C8769D32C012C852068222E59
:100EC000830123FC19C0832D90E048165906A0F435
:100ED000B70180E290E06FD33A94F5CFF50127FC9B
:100EE000859127FE81915F01B70190E064D33110B5
:100EF0003A94F1E04F1A51084114510479F7DEC0D9
:100F0000843611F0893631F5F80127FF07C060817A
:100F10007181828193810C5F1F4F08C06081718154
:100F2000882777FD8095982F0E5F1F4F2F76B22E62
:100F300097FF09C090958095709561957F4F8F4F71
:100F40009F4F2068B22E2AE030E0A40166D3A82E7D
:100F5000A81843C0853729F42F7EB22E2AE030E04E
:100F600025C0F22FF97FBF2E8F36C1F018F48835D7
:100F700079F0ADC0803719F0883721F0A8C02F2F45
:100F80002061B22EB4FE0DC08B2D8460B82E09C036
:100F900024FF0AC09F2F9660B92E06C028E030E0DB
:100FA00005C020E130E002C020E132E0F801B7FEE8
:100FB00007C060817181828193810C5F1F4F06C0E1
:100FC0006081718180E090E00E5F1F4FA40125D306
:100FD000A82EA818FB2DFF77BF2EB6FE0BC02B2D19
:100FE0002E7FA51450F4B4FE0AC0B2FC08C02B2D0D
:100FF0002E7E05C07A2C2B2D03C07A2C01C0752CB7
:1010000024FF0DC0FE01EA0DF11D8081803311F433
:10101000297E09C022FF06C07394739404C0822FF6
:10102000867809F0739423FD12C020FF06C05A2C65
:10103000731418F4530C5718732C731460F4B7011D
:1010400080E290E02C87B7D273942C85F6CF73148E
:1010500010F4371801C0312C24FF11C0B70180E310
:1010600090E02C87A8D22C8522FF16C021FF03C058
:1010700088E590E002C088E790E0B7010CC0822FBD
:10108000867851F021FD02C080E201C08BE227FD8D
:101090008DE2B70190E08FD2A51430F4B70180E360
:1010A00090E089D25A94F8CFAA94F401EA0DF11D88
:1010B0008081B70190E07FD2A110F6CF332009F4F0
:1010C0005DCEB70180E290E076D23A94F7CFF70197
:1010D0008681978102C08FEF9FEF2C96E2E117C3C4
:1010E0006F927F929F92AF92BF92CF92DF92EF92D8
:1010F000FF920F931F93CF93DF93CDB7DEB729975E
:101100000FB6F894DEBF0FBECDBF6A01B22E102F0E
:101110000C3320F4FF24F394F00E02C04CE3F42EC1
:101120000F2D27E0AE014F5F5F4F57D17981272FF9
:101130002970213031F0E1FC06C0E0FC06C060E01F
:1011400005C06DE203C06BE201C060E2AE2DA0718C
:1011500073FF36C0662311F084E001C083E08B1575
:1011600010F4B81A01C0B12CA1110BC0F6018B2DDF
:1011700090E2882319F091938150FBCFCB0CD11CC6
:10118000B12C662331F0F601608396012F5F3F4F4B
:101190006901C6010396E2FE05C02EE4F601208334
:1011A00031E404C02EE6F601208331E63183228348
:1011B000FC012B2D30E22223F1F131932150FBCFA2
:1011C00072FF40C0662311F084E001C083E08B15FC
:1011D00010F4B81A01C0B12CA1110BC0F6018B2D6F
:1011E00090E2882319F091938150FBCFCB0CD11C56
:1011F000B12C662331F0F601608396012F5F3F4FDB
:101200006901C6010396E2FE07C029E4F6012083C6
:101210002EE4218326E406C029E6F60120832EE68B
:10122000218326E62283FC012B2D30E2222319F0B4
:1012300031932150FBCFFC01EB0DF11D10828EEF9D
:101240009FEFB7C0B1E0611101C0B0E04B2F50E09B
:101250001816190624F49C012F5F3F4F02C021E0AD
:1012600030E0240F351F112329F0412F50E04F5F4C
:101270005F4F02C040E050E0420F531F2B2D30E083
:101280004217530714F4B41A01C0B12C2E2D287143
:1012900059F4F6012B2D30E2222319F0319321501D
:1012A000FBCFCB0CD11CB12CBB2331F0F6016083FA
:1012B00096012F5F3F4F6901A1110BC0F6012B2D45
:1012C00030E3222319F031932150FBCFCB0CD11CFA
:1012D000B12CF80E0A81372F3071A32E74FF03C092
:1012E000013309F4FA941F142CF42F2D293018F02F
:1012F00028E001C021E0682F392F97FF02C060E08D
:1013000030E0462F532F612C712C3EE2932EBC010E
:10131000621B71099B01DC01A41BB50BE1E0F0E04D
:10132000EC0FFD1FAE0FBF1FE12EF12CF194E194E5
:10133000F1084F3FFFEF5F0731F4F6019082B601ED
:101340006F5F7F4F6B01841795074CF024173507AB
:1013500034F4BD01660D771DFB01118101C010E35E
:1013600041505109FFEF6F1A7F0AB6016F5F7F4F3F
:101370004E155F0524F0F60110836B01DACF481794
:10138000590739F4063320F4053319F4A11001C0CC
:1013900011E3F6011083FB018B2D90E2882319F0F5
:1013A00091938150FBCFFB01EB0DF11D108280E08A
:1013B00090E029960FB6F894DEBF0FBECDBFDF9147
:1013C000CF911F910F91FF90EF90DF90CF90BF9042
:1013D000AF909F907F906F900895283008F027E09D
:1013E0003327DA01990F311D87FD91600096610561
:1013F000710539F432602E5F3D9330E32A95E1F7B1
:1014000008959F3F30F080387105610509F03C5F19
:101410003C5F3D93913008F08068911DDF93CF933E
:101420001F930F93FF92EF92192F987F9695E92FB4
:1014300096959695E90FFF27EE53FF4F992733278F
:10144000EE24FF24A701E70105900894079428F4EF
:10145000360FE71EF81E491F511D660F771F881FA4
:10146000991F0694A1F70590079428F4E70EF81E3B
:10147000491F561FC11D770F881F991F661F0694AD
:10148000A1F70590079428F4F80E491F561FC71FAF
:10149000D11D880F991F661F771F0694A1F705902D
:1014A000079420F4490F561FC71FD81F990F661FB6
:1014B000771F881F0694A9F784911095177041F043
:1014C000D695C79557954795F794E7941A95C1F720
:1014D000E8E6F0E068941590159135916591959145
:1014E00005907FE27395E118F10A430B560BC90B87
:1014F000D009C0F7E10CF11E431F561FC91FD01DB4
:101500007EF4703311F48A95E6CFE894015030F000
:10151000080F0AF40027021708F4202F2395022F42
:101520007A3328F079E37D932A95E9F710C07D930B
:101530002A9589F606949795679537951795179488
:10154000E118F10A430B560BC90BD00998F023950B
:101550007E9173957A3308F070E37C932013B8F78B
:101560007E9170617D9330F0839571E37D9370E39C
:101570002A95E1F71124EF90FF900F911F91CF91E1
:10158000DF91992787FD90950895FC0105906150A2
:1015900070400110D8F7809590958E0F9F1F089589
:1015A000FC016150704001900110D8F78095909532
:1015B0008E0F9F1F08950F931F93CF93DF93182FC4
:1015C000092FEB018B8181FD03C08FEF9FEF20C0BE
:1015D00082FF10C04E815F812C813D8142175307ED
:1015E0007CF4E881F9819F012F5F3F4F3983288385
:1015F000108306C0E885F985812F0995892B29F785
:101600002E813F812F5F3F4F3F832E83812F902F6D
:10161000DF91CF911F910F910895FA01AA272830E9
:1016200051F1203181F1E8946F936E7F6E5F7F4FAF
:101630008F4F9F4FAF4FB1E03ED0B4E03CD0670F2B
:10164000781F891F9A1FA11D680F791F8A1F911D7E
:10165000A11D6A0F711D811D911DA11D20D009F4CE
:1016600068943F912AE0269F11243019305D319310
:10167000DEF6CF010895462F4770405D4193B3E0F9
:101680000FD0C9F7F6CF462F4F70405D4A3318F0A0
:10169000495D31FD4052419302D0A9F7EACFB4E051
:1016A000A6959795879577956795BA95C9F7009709
:1016B0006105710508959B01AC010A2E06945795AA
:1016C000479537952795BA95C9F7620F731F841F01
:1016D000951FA01D08952F923F924F925F926F9297
:1016E0007F928F929F92AF92BF92CF92DF92EF92B2
:1016F000FF920F931F93CF93DF93CDB7DEB7CA1B33
:10170000DB0B0FB6F894DEBF0FBECDBF09942A885D
:10171000398848885F846E847D848C849B84AA8405
:10172000B984C884DF80EE80FD800C811B81AA8192
:10173000B981CE0FD11D0FB6F894DEBF0FBECDBF5D
:08174000ED010895F894FFCFBC
:101748005469202533642043202564202020546FC9
:101758002025336420432025640D0A004C2025737E
:101768002020282573290D0A004D616765720049FC
:101778006465616C00466574742100040000000013
:101788004005003333F33F06006666E63F08009ADB
:1017980099D93F0A00CDCCCC3F0C000000C03F0FC8
:1017A800003333B33F14006666A63F1C009A99992C
:1017B8003F2800CDCC8C3F44003333833F90010059
:1017C80000803F200348E17A3F5C036666663F700D
:0617D80003CDCC4C3F00E4
:00000001FF
